:10503C0033302E322020200006012C034D056E0744
:10504C008F09A70B0000000000000032006400C8AC
:10505C00012C015E019001C201FC022E026102943E
:10506C0002C702FA032C035F039203C503F8042A58
:10507C00045D049004C304F60528055B058E05C188
:10508C0005F406260659068C06BF06F207240757B8
:10509C00078A07BD07F008220855088808BB08EEE8
:1050AC0009210953098609B909EC0A1F0A510A8416
:1050BC000AB70AEA0B1D0B4F0B820BB50BE80C1B46
:1050CC000C4D0C800CB30CE60D190D4B0D7E0DB177
:1050DC000DE40E170E490E7C0EAF0EE20F150F47A6
:1050EC000F7A0FAD0FE010131045107810AB10DED7
:1050FC0011111144117611A911DC120F1242127404
:10510C0012A712DA130D1340137213A513D8140B34
:10511C00143E147014A314D61509153C156E15A164
:10512C0015D41607163A166C169F16D21705173893
:10513C00176A179D17D0180318361868189B18CEC5
:10514C00190119341967199919CC19FF1A321A65F2
:10515C001A971ACA1AFD1B301B631B951BC81BFB25
:10516C001C2E1C611C931CC61CF91D2C1D5F1D9153
:10517C001DC41DF71E2A1E5D1E8F1EC21EF51F2884
:10518C001F5B1F8D1FC01FF320262059208B20BEB4
:10519C0020F121242157218921BC21EF22222255E3
:1051AC00228822BA22ED23202353238623B823EB13
:1051BC00241E2451248424B624E9251C254F258241
:1051CC0025B425E7261A264D268026B226E5271873
:1051DC00274B277E27B027E328162849287C28AEA2
:1051EC0028E129142947297A29AC29DF2A122A45D2
:1051FC002A782AAB2ADD2B102B432B762BA92BDB01
:10520C002C0E2C412C742CA72CD92D0C2D3F2D722F
:10521C002DA52DD72E0A2E3D2E702EA32ED52F0860
:10522C002F3B2F6E2FA12FD330063039306C309F8F
:10523C0030D131043137316A319D31CF32023235C0
:10524C003268329B32CE330033333366339933CCEE
:10525C0033FE34313464349734CA34FC352F356220
:10526C00359535C835FA362D3660369336C636F850
:10527C00372B375E379137C437F63829385C388F7F
:10528C0038C238F43927395A398D39C039F23A25B0
:10529C003A583A8B3ABE3AF03B233B563B893BBCDF
:1052AC003BEF3C213C543C873CBA3CED3D1F3D520E
:1052BC003D853DB83DEB3E1D3E503E833EB63EE93E
:1052CC003F1B3F4E3F813FB43FE74019404C407F6E
:1052DC0040B240E54117414A417D41B041E342159E
:1052EC004248427B42AE42E143134346437943ACCE
:1052FC0043DF44124444447744AA44DD45104542FC
:10530C00457545A845DB460E4640467346A646D92C
:10531C00470C473E477147A447D7480A483C486F5B
:10532C0048A248D54908493A496D49A049D34A068B
:10533C004A384A6B4A9E4AD14B044B364B694B9CBC
:10534C004BCF4C024C354C674C9A4CCD4D004D33E9
:10535C004D654D984DCB4DFE4E314E634E964EC91C
:10536C004EFC4F2F4F614F944FC74FFA502D505F4B
:10537C00509250C550F8512B515D519051C351F67C
:10538C005229525B528E52C152F453275359538CAB
:10539C0053BF53F254255457548A54BD54F05523DB
:1053AC005556558855BB55EE56215654568656B90A
:1053BC0056EC571F5752578457B757EA581D585039
:1053CC00588258B558E8591B594E598059B359E66B
:1053DC005A195A4C5A7E5AB15AE45B175B4A5B7C99
:1053EC005BAF5BE25C155C485C7A5CAD5CE05D13CA
:1053FC005D465D795DAB5DDE5E115E445E775EA9F8
:10540C005EDC5F0F5F425F755FA75FDA600D604027
:10541C00607360A560D8610B613E617161A361D658
:10542C006209623C626F62A162D46307633A636D86
:10543C00639F63D264056438646B649D64D06503B8
:10544C0065366569659B65A765B265BD65C865D33D
:10545C0065DE65E965F465FF660A66156620662BF0
:10546C0066366641664C66576662666D667866831C
:10547C00668E669966A466AF66BA66C566D066DB4C
:10548C0066E666F166FC67086713671E6729673472
:10549C00673F674A67556760676B67766781678C9C
:1054AC00679767A267AD67B867C367CE67D967E4CC
:1054BC0067EF67FA68056810681B68266831683CF6
:1054CC0068476852685D68686874687F688A689520
:1054DC0068A068AB68B668C168CC68D768E268ED4C
:1054EC0068F86903690E69196924692F693A694575
:1054FC006950695B69666971697C69876992699DA4
:10550C0069A869B369BE69C969D569E069EB69F6CF
:10551C006A016A0C6A176A226A2D6A386A436A4EF3
:10552C006A596A646A6F6A7A6A856A906A9B6AA623
:10553C006AB16ABC6AC76AD26ADD6AE86AF36AFE53
:10554C006B096B146B1F6B2A6B356B416B4C6B5778
:10555C006B626B6D6B786B836B8E6B996BA46BAFA3
:10556C006BBA6BC56BD06BDB6BE66BF16BFC6C07D2
:10557C006C126C1D6C286C336C3E6C496C546C5FFB
:10558C006C6A6C756C806C8B6C966CA26CAD6CB828
:10559C006CC36CCE6CD96CE46CEF6CFA6D056D1051
:1055AC006D1B6D266D316D3C6D476D526D5D6D687B
:1055BC006D736D7E6D896D946D9F6DAA6DB56DC0AB
:1055CC006DCB6DD66DE16DEC6DF76E026E0E6E19D6
:1055DC006E246E2F6E3A6E456E506E5B6E666E71FB
:1055EC006E7C6E876E926E9D6EA86EB36EBE6EC92B
:1055FC006ED46EDF6EEA6EF56F006F0B6F166F2157
:10560C006F2C6F376F426F4D6F586F636F6E6F7A81
:10561C006F856F906F9B6FA66FB16FBC6FC76FD2AA
:10562C006FDD6FE86FF36FFE70097014701F702AD6
:10563C0070357040704B70567061706C7077708202
:10564C00708D709870A370AE70B970C470CF70DB31
:10565C0070E670F170FC71077112711D7128713355
:10566C00713E71497154715F716A71757180718B82
:10567C00719671A171AC71B771C271CD71D871E3B2
:10568C0071EE71F97204720F721A72257230723BDC
:10569C0072477252725D72687273727E7289729402
:1056AC00729F72AA72B572C072CB72D672E172EC32
:1056BC0072F77302730D73187323732E733973445B
:1056CC00734F735A73657370737B73867391739C8A
:1056DC0073A873B373BE73C973D473DF73EA73F5B2
:1056EC007400740B74167421742C74377442744DDA
:1056FC0074587463746E74797484748F749A74A50A
:10570C0074B074BB74C674D174DC74E774F274FD39
:10571C0075087514751F752A75357540754B75565A
:10572C007561756C75777582758D759875A375AE89
:10573C0075B975C475CF75DA75E575F075FB7606B8
:10574C007611761C76277632763D76487653765EE1
:10575C00766976757680768B769676A176AC76B70A
:10576C0076C276CD76D876E376EE76F97704770F37
:10577C00771A77257730773B77467751775C776761
:10578C007772777D77887793779E77A977B477BF91
:10579C0077CA77D577E177EC77F77802780D7818B8
:1057AC007823782E78397844784F785A78657870E1
:1057BC00787B78867891789C78A778B278BD78C811
:1057CC0078D378DE78E978F478FF790A791579203E
:1057DC00792B79367941794D79587963796E797964
:1057EC007984798F799A79A579B079BB79C679D191
:1057FC0079DC79E779F279FD7A087A137A1E7A29BD
:10580C007A347A3F7A4A7A557A607A6B7A767A81E8
:10581C007A8C7A977AA27AAE7AB97AC47ACF7ADA13
:10582C007AE57AF07AFB7B067B117B1C7B277B323B
:10583C007B3D7B487B537B5E7B697B747B7F7B8A68
:10584C007B957BA07BAB7BB67BC17BCC7BD77BE298
:10585C007BED7BF87C037C0E7C1A7C257C307C3BBE
:10586C007C467C517C5C7C677C727C7D7C887C93E8
:10587C007C9E7CA97CB47CBF7CCA7CD57CE07CEB18
:10588C007CF67D017D0C7D177D227D2D7D387D4341
:10589C007D4E7D597D647D6F7D7B7D867D917D9C6C
:1058AC007DA77DB27DBD7DC87DD37DDE7DE97DF498
:1058BC007DFF7E0A7E157E207E2B7E367E417E4CC1
:1058CC007E577E627E6D7E787E837E8E7E997EA4F0
:1058DC007EAF7EBA7EC57ED07EDB7EE77EF27EFD1D
:1058EC007F087F137F1E7F297F347F3F7F4A7F5540
:1058FC007F607F6B7F767F817F8C7F977FA27FAD70
:10590C007FB87FC37FCE7FD97FE47FEF7FFA80059E
:10591C008010801B80268031803C80488053805EC4
:10592C0080698074807F808A809580A080AB80B6EF
:10593C0080C180CC80D780E280ED80F88103810E1D
:10594C0081198124812F813A81458150815B816647
:10595C008171817C81878192819D81A881B481BF75
:10596C0081CA81D581E081EB81F68201820C82179C
:10597C008222822D82388243824E82598264826FC7
:10598C00827A82858290829B82A682B182BC82C7F7
:10599C0082D282DD82E882F382FE83098314832023
:1059AC00832B83368341834C83578362836D837847
:1059BC008383838E839983A483AF83BA83C583D077
:1059CC0083DB83E683F183FC84078412841D8428A3
:1059DC008433843E84498454845F846A84758481CE
:1059EC00848C849784A284AD84B884C384CE84D9F7
:1059FC0084E484EF84FA85058510851B8526853122
:105A0C00853C85478552855D85688573857E85894E
:105A1C008594859F85AA85B585C085CB85D685E17E
:105A2C0085ED85F88603860E86198624862F863AA0
:105A3C0086458650865B86668671867C86878692CE
:105A4C00869D86A886B386BE86C986D486DF86EAFE
:105A5C0086F58700870B87168721872C8737874227
:105A6C00874E87598764876F877A87858790879B4E
:105A7C0087A687B187BC87C787D287DD87E887F37E
:105A8C0087FE88098814881F882A88358840884BA7
:105A9C0088568861886C88778882888D889888A3D6
:105AAC0088AE88BA88C588D088DB88E688F188FCFF
:105ABC0089078912891D89288933893E8949895426
:105ACC00895F896A89758980898B899689A189AC56
:105ADC0089B789C289CD89D889E389EE89F98A0485
:105AEC008A0F8A1B8A268A318A3C8A478A528A5DA7
:105AFC008A688A738A7E8A898A948A9F8AAA8AB5D6
:105B0C008AC08ACB8AD68AE18AEC8AF78B028B0D03
:105B1C008B188B238B2E8B398B448B4F8B5A8B652D
:105B2C008B708B7B8B878B928B9D8BA88BB38BBE57
:105B3C008BC98BD48BDF8BEA8BF58C008C0B8C1682
:105B4C008C218C2C8C378C428C4D8C588C638C6EAD
:105B5C008C798C848C8F8C9A8CA58CB08CBB8CC6DD
:105B6C008CD18CDC8CE78CF38CFE8D098D148D1F05
:105B7C008D2A8D358D408D4B8D568D618D6C8D772D
:105B8C008D828D8D8D988DA38DAE8DB98DC48DCF5D
:105B9C008DDA8DE58DF08DFB8E068E118E1C8E2789
:105BAC008E328E3D8E488E548E5F8E6A8E758E80B0
:105BBC008E8B8E968EA18EAC8EB78EC28ECD8ED8DD
:105BCC008EE38EEE8EF98F048F0F8F1A8F258F3008
:105BDC008F3B8F468F518F5C8F678F728F7D8F8835
:105BEC008F938F9E8FA98FB48FC08FCB8FD68FE161
:105BFC008FEC8FF79002900D90189023902E903987
:105C0C009044904F905A90659070907B90869091B4
:105C1C00909C90A790B290BD90C890D390DE90E9E4
:105C2C0090F490FF910A91159121912C913791420A
:105C3C00914D91589163916E91799184918F919A34
:105C4C0091A591B091BB91C691D191DC91E791F264
:105C5C0091FD92089213921E92299234923F924A8D
:105C6C0092559260926B92769281928D929892A3B9
:105C7C0092AE92B992C492CF92DA92E592F092FBE4
:105C8C0093069311931C93279332933D934893530C
:105C9C00935E93699374937F938A939593A093AB3C
:105CAC0093B693C193CC93D793E293EE93F9940468
:105CBC00940F941A94259430943B94469451945C8C
:105CCC0094679472947D94889493949E94A994B4BC
:105CDC0094BF94CA94D594E094EB94F69501950CEA
:105CEC0095179522952D95389543954E955A956512
:105CFC009570957B95869591959C95A795B295BD3C
:105D0C0095C895D395DE95E995F495FF960A961569
:105D1C009620962B96369641964C96579662966D93
:105D2C0096789683968E969996A496AF96BA96C6C2
:105D3C0096D196DC96E796F296FD97089713971EE8
:105D4C0097299734973F974A97559760976B977613
:105D5C009781978C979797A297AD97B897C397CE43
:105D6C0097D997E497EF97FA98059810981B98276E
:105D7C009832983D98489853985E98699874987F93
:105D8C00988A989598A098AB98B698C198CC98D7C3
:105D9C0098E298ED98F89903990E99199924992FEE
:105DAC00993A99459950995B99669971997C99871B
:105DBC009993999E99A999B499BF99CA99D599E043
:105DCC0099EB99F69A019A0C9A179A229A2D9A386D
:105DDC009A439A4E9A599A649A6F9A7A9A859A909B
:105DEC009A9B9AA69AB19ABC9AC79AD29ADD9AE8CB
:105DFC009AF49AFF9B0A9B159B209B2B9B369B41ED
:105E0C009B4C9B579B629B6D9B789B839B8E9B991A
:105E1C009BA49BAF9BBA9BC59BD09BDB9BE69BF14A
:105E2C009BFC9C079C129C1D9C289C339C3E9C4973
:105E3C009C549C609C6B9C769C819C8C9C979CA29B
:105E4C009CAD9CB89CC39CCE9CD99CE49CEF9CFACA
:105E5C009D059D109D1B9D269D319D3C9D479D52F2
:105E6C009D5D9D689D739D7E9D899D949D9F9DAA22
:105E7C009DB59DC19DCC9DD79DE29DED9DF89E034A
:105E8C009E0E9E199E249E2F9E3A9E459E509E5B72
:105E9C009E669E719E7C9E879E929E9D9EA89EB3A2
:105EAC009EBE9EC99ED49EDF9EEA9EF59F009F0BD0
:105EBC009F169F219F2D9F389F439F4E9F599F64F4
:105ECC009F6F9F7A9F859F909F9B9FA69FB19FBC22
:105EDC009FC79FD29FDD9FE89FF39FFEA009A01450
:105EEC00A01FA02AA035A040A04BA056A061A06C7A
:105EFC00A077A082A08DA099A0A4A0AFA0BAA0C5A5
:105F0C00A0D0A0DBA0E6A0F1A0FCA107A112A11DCE
:105F1C00A128A133A13EA149A154A15FA16AA175F9
:105F2C00A180A18BA196A1A1A1ACA1B7A1C2A1CD29
:105F3C00A1D8A1E3A1EEA1FAA205A210A21BA22650
:105F4C00A231A23CA247A252A25DA268A273A27E79
:105F5C00A289A294A29FA2AAA2B5A2C0A2CBA2D6A9
:105F6C00A2E1A2ECA2F7A302A30DA318A323A32ED4
:105F7C00A339A344A34FA35AA366A371A37CA387FD
:105F8C00A392A39DA3A8A3B3A3BEA3C9A3D4A3DF29
:105F9C00A3EAA3F5A400A40BA416A421A42CA43753
:105FAC00A442A44DA458A463A46EA479A484A48F81
:105FBC00A49AA4A5A4B0A4BBA4C7A4D2A4DDA4E8AD
:105FCC00A4F3A4FEA509A514A51FA52AA535A540D3
:105FDC00A54BA556A561A56CA577A582A58DA59801
:105FEC00A5A3A5AEA5B9A5C4A5CFA5DAA5E5A5F031
:105FFC00A5FBA606A611A61CA627A633A63EA64957
:10600C00A654A65FA66AA675A680A68BA696A6A180
:10601C00A6ACA6B7A6C2A6CDA6D8A6E3A6EEA6F9B0
:10602C00A704A70FA71AA725A730A73BA746A751D8
:10603C00A75CA767A772A77DA788A794A79FA7AA05
:10604C00A7B5A7C0A7CBA7D6A7E1A7ECA7F7A8022F
:10605C00A80DA818A823A82EA839A844A84FA85A58
:10606C00A865A870A87BA886A891A89CA8A7A8B288
:10607C00A8BDA8C8A8D3A8DEA8E9A8F4A900A90BB4
:10608C00A916A921A92CA937A942A94DA958A963D8
:10609C00A96EA979A984A98FA99AA9A5A9B0A9BB08
:1060AC00A9C6A9D1A9DCA9E7A9F2A9FDAA08AA1336
:1060BC00AA1EAA29AA34AA3FAA4AAA55AA60AA6C5F
:1060CC00AA77AA82AA8DAA98AAA3AAAEAAB9AAC488
:1060DC00AACFAADAAAE5AAF0AAFBAB06AB11AB1CB5
:1060EC00AB27AB32AB3DAB48AB53AB5EAB69AB74E0
:1060FC00AB7FAB8AAB95ABA0ABABABB6ABC1ABCD0F
:10610C00ABD8ABE3ABEEABF9AC04AC0FAC1AAC2533
:10611C00AC30AC3BAC46AC51AC5CAC67AC72AC7D5F
:10612C00AC88AC93AC9EACA9ACB4ACBFACCAACD58F
:10613C00ACE0ACEBACF6AD01AD0CAD17AD22AD2DBA
:10614C00AD39AD44AD4FAD5AAD65AD70AD7BAD86DF
:10615C00AD91AD9CADA7ADB2ADBDADC8ADD3ADDE0F
:10616C00ADE9ADF4ADFFAE0AAE15AE20AE2BAE363A
:10617C00AE41AE4CAE57AE62AE6DAE78AE83AE8E67
:10618C00AE9AAEA5AEB0AEBBAEC6AED1AEDCAEE78F
:10619C00AEF2AEFDAF08AF13AF1EAF29AF34AF3FB9
:1061AC00AF4AAF55AF60AF6BAF76AF81AF8CAF97E7
:1061BC00AFA2AFADAFB8AFC3AFCEAFD9AFE4AFEF17
:1061CC00AFFAB006B011B01CB027B032B03DB04839
:1061DC00B053B05EB069B074B07FB08AB095B0A067
:1061EC00B0ABB0B6B0C1B0CCB0D7B0E2B0EDB0F897
:1061FC00B103B10EB119B124B12FB13AB145B150BF
:10620C00B15BB167B172B17DB188B193B19EB1A9E7
:10621C00B1B4B1BFB1CAB1D5B1E0B1EBB1F6B20115
:10622C00B20CB217B222B22DB238B243B24EB2593E
:10623C00B264B26FB27AB285B290B29BB2A6B2B16E
:10624C00B2BCB2C7B2D3B2DEB2E9B2F4B2FFB30A97
:10625C00B315B320B32BB336B341B34CB357B362BE
:10626C00B36DB378B383B38EB399B3A4B3AFB3BAEE
:10627C00B3C5B3D0B3DBB3E6B3F1B3FCB407B4121C
:10628C00B41DB428B433B43FB44AB455B460B46B41
:10629C00B476B481B48CB497B4A2B4ADB4B8B4C36E
:1062AC00B4CEB4D9B4E4B4EFB4FAB505B510B51B9B
:1062BC00B526B531B53CB547B552B55DB568B573C6
:1062CC00B57EB589B594B5A0B5ABB5B6B5C1B5CCF1
:1062DC00B5D7B5E2B5EDB5F8B603B60EB619B6241A
:1062EC00B62FB63AB645B650B65BB666B671B67C46
:1062FC00B687B692B69DB6A8B6B3B6BEB6C9B6D476
:10630C00B6DFB6EAB6F5B700B70CB717B722B72D9C
:10631C00B738B743B74EB759B764B76FB77AB785C5
:10632C00B790B79BB7A6B7B1B7BCB7C7B7D2B7DDF5
:10633C00B7E8B7F3B7FEB809B814B81FB82AB83520
:10634C00B840B84BB856B861B86DB878B883B88E49
:10635C00B899B8A4B8AFB8BAB8C5B8D0B8DBB8E675
:10636C00B8F1B8FCB907B912B91DB928B933B93E9F
:10637C00B949B954B95FB96AB975B980B98BB996CD
:10638C00B9A1B9ACB9B7B9C2B9CDB9D9B9E4B9EFFA
:10639C00B9FABA05BA10BA1BBA26BA31BA3CBA471E
:1063AC00BA52BA5DBA68BA73BA7EBA89BA94BA9F4D
:1063BC00BAAABAB5BAC0BACBBAD6BAE1BAECBAF77D
:1063CC00BB02BB0DBB18BB23BB2EBB3ABB45BB50A2
:1063DC00BB5BBB66BB71BB7CBB87BB92BB9DBBA8CD
:1063EC00BBB3BBBEBBC9BBD4BBDFBBEABBF5BC00FC
:1063FC00BC0BBC16BC21BC2CBC37BC42BC4DBC5825
:10640C00BC63BC6EBC79BC84BC8FBC9ABCA6BCB152
:10641C00BCBCBCC7BCD2BCDDBCE8BCF3BCFEBD097B
:10642C00BD14BD1FBD2ABD35BD40BD4BBD56BD61A4
:10643C00BD6CBD77BD82BD8DBD98BDA3BDAEBDB9D4
:10644C00BDC4BDCFBDDABDE5BDF0BDFBBE06BE1201
:10645C00BE1DBE28BE33BE3EBE49BE54BE5FBE6A24
:10646C00BE75BE80BE8BBE96BEA1BEACBEB7BEC254
:10647C00BECDBED8BEE3BEEEBEF9BF04BF0FBF1A81
:10648C00BF25BF30BF3BBF46BF51BF5CBF67BF73AB
:10649C00BF7EBF89BF94BF9FBFAABFB5BFC0BFCBD4
:1064AC00BFD6BFE1BFECBFF7C002C00DC018C02300
:1064BC00C02EC039C044C04FC05AC065C070C07B2C
:1064CC00C086C091C09CC0A7C0B2C0BDC0C8C0D35C
:1064DC00C0DFC0EAC0F5C100C10BC116C121C12C7F
:1064EC00C137C142C14DC158C163C16EC179C184AC
:1064FC00C18FC19AC1A5C1B0C1BBC1C6C1D1C1DCDC
:10650C00C1E7C1F2C1FDC208C213C21EC229C23406
:10651C00C240C24BC256C261C26CC277C282C28D2B
:10652C00C298C2A3C2AEC2B9C2C4C2CFC2DAC2E55B
:10653C00C2F0C2FBC306C311C31CC327C332C33D85
:10654C00C348C353C35EC369C374C37FC38AC395B3
:10655C00C3A0C3ACC3B7C3C2C3CDC3D8C3E3C3EEDC
:10656C00C3F9C404C40FC41AC425C430C43BC44604
:10657C00C451C45CC467C472C47DC488C493C49E33
:10658C00C4A9C4B4C4BFC4CAC4D5C4E0C4EBC4F663
:10659C00C501C50DC518C523C52EC539C544C54F84
:1065AC00C55AC565C570C57BC586C591C59CC5A7B3
:1065BC00C5B2C5BDC5C8C5D3C5DEC5E9C5F4C5FFE3
:1065CC00C60AC615C620C62BC636C641C64CC6570B
:1065DC00C662C66DC679C684C68FC69AC6A5C6B035
:1065EC00C6BBC6C6C6D1C6DCC6E7C6F2C6FDC70862
:1065FC00C713C71EC729C734C73FC74AC755C7608B
:10660C00C76BC776C781C78CC797C7A2C7ADC7B8BA
:10661C00C7C3C7CEC7D9C7E5C7F0C7FBC806C811E3
:10662C00C81CC827C832C83DC848C853C85EC8690A
:10663C00C874C87FC88AC895C8A0C8ABC8B6C8C13A
:10664C00C8CCC8D7C8E2C8EDC8F8C903C90EC91967
:10665C00C924C92FC93AC946C951C95CC967C9728D
:10666C00C97DC988C993C99EC9A9C9B4C9BFC9CABA
:10667C00C9D5C9E0C9EBC9F6CA01CA0CCA17CA22E6
:10668C00CA2DCA38CA43CA4ECA59CA64CA6FCA7A12
:10669C00CA85CA90CA9BCAA6CAB2CABDCAC8CAD33E
:1066AC00CADECAE9CAF4CAFFCB0ACB15CB20CB2B66
:1066BC00CB36CB41CB4CCB57CB62CB6DCB78CB8392
:1066CC00CB8ECB99CBA4CBAFCBBACBC5CBD0CBDBC2
:1066DC00CBE6CBF1CBFCCC07CC13CC1ECC29CC34E9
:1066EC00CC3FCC4ACC55CC60CC6BCC76CC81CC8C12
:1066FC00CC97CCA2CCADCCB8CCC3CCCECCD9CCE442
:10670C00CCEFCCFACD05CD10CD1BCD26CD31CD3C6B
:10671C00CD47CD52CD5DCD68CD73CD7FCD8ACD9596
:10672C00CDA0CDABCDB6CDC1CDCCCDD7CDE2CDEDC1
:10673C00CDF8CE03CE0ECE19CE24CE2FCE3ACE45EA
:10674C00CE50CE5BCE66CE71CE7CCE87CE92CE9D19
:10675C00CEA8CEB3CEBECEC9CED4CEE0CEEBCEF646
:10676C00CF01CF0CCF17CF22CF2DCF38CF43CF4E69
:10677C00CF59CF64CF6FCF7ACF85CF90CF9BCFA699
:10678C00CFB1CFBCCFC7CFD2CFDDCFE8CFF3CFFEC9
:10679C00D009D014D01FD02AD035D040D04CD057EF
:1067AC00D062D06DD078D083D08ED099D0A4D0AF19
:1067BC00D0BAD0C5D0D0D0DBD0E6D0F1D0FCD10748
:1067CC00D112D11DD128D133D13ED149D154D15F71
:1067DC00D16AD175D180D18BD196D1A1D1ACD1B8A0
:1067EC00D1C3D1CED1D9D1E4D1EFD1FAD205D210C7
:1067FC00D21BD226D231D23CD247D252D25DD268F1
:10680C00D273D27ED289D294D29FD2AAD2B5D2C020
:10681C00D2CBD2D6D2E1D2ECD2F7D302D30DD3194C
:10682C00D324D32FD33AD345D350D35BD366D37170
:10683C00D37CD387D392D39DD3A8D3B3D3BED3C9A0
:10684C00D3D4D3DFD3EAD3F5D400D40BD416D421CC
:10685C00D42CD437D442D44DD458D463D46ED479F8
:10686C00D485D490D49BD4A6D4B1D4BCD4C7D4D220
:10687C00D4DDD4E8D4F3D4FED509D514D51FD52A4C
:10688C00D535D540D54BD556D561D56CD577D58278
:10689C00D58DD598D5A3D5AED5B9D5C4D5CFD5DAA8
:1068AC00D5E6D5F1D5FCD607D612D61DD628D633CB
:1068BC00D63ED649D654D65FD66AD675D680D68BF8
:1068CC00D696D6A1D6ACD6B7D6C2D6CDD6D8D6E328
:1068DC00D6EED6F9D704D70FD71AD725D730D73B52
:1068EC00D746D752D75DD768D773D77ED789D79479
:1068FC00D79FD7AAD7B5D7C0D7CBD7D6D7E1D7ECA8
:10690C00D7F7D802D80DD818D823D82ED839D844D0
:10691C00D84FD85AD865D870D87BD886D891D89CFF
:10692C00D8A7D8B3D8BED8C9D8D4D8DFD8EAD8F528
:10693C00D900D90BD916D921D92CD937D942D94D4F
:10694C00D958D963D96ED979D984D98FD99AD9A57F
:10695C00D9B0D9BBD9C6D9D1D9DCD9E7D9F2D9FDAF
:10696C00DA08DA13DA1FDA2ADA35DA40DA4BDA56D1
:10697C00DA61DA6CDA77DA82DA8DDA98DAA3DAAEFF
:10698C00DAB9DAC4DACFDADADAE5DAF0DAFBDB062E
:10699C00DB11DB1CDB27DB32DB3DDB48DB53DB5E57
:1069AC00DB69DB74DB7FDB8BDB96DBA1DBACDBB782
:1069BC00DBC2DBCDDBD8DBE3DBEEDBF9DC04DC0FAD
:1069CC00DC1ADC25DC30DC3BDC46DC51DC5CDC67D7
:1069DC00DC72DC7DDC88DC93DC9EDCA9DCB4DCBF07
:1069EC00DCCADCD5DCE0DCECDCF7DD02DD0DDD182F
:1069FC00DD23DD2EDD39DD44DD4FDD5ADD65DD7057
:106A0C00DD7BDD86DD91DD9CDDA7DDB2DDBDDDC886
:106A1C00DDD3DDDEDDE9DDF4DDFFDE0ADE15DE20B3
:106A2C00DE2BDE36DE41DE4CDE58DE63DE6EDE79DA
:106A3C00DE84DE8FDE9ADEA5DEB0DEBBDEC6DED106
:106A4C00DEDCDEE7DEF2DEFDDF08DF13DF1EDF2932
:106A5C00DF34DF3FDF4ADF55DF60DF6BDF76DF815E
:106A6C00DF8CDF97DFA2DFADDFB9DFC4DFCFDFDA8A
:106A7C00DFE5DFF0DFFBE006E011E01CE027E032B1
:106A8C00E03DE048E053E05EE069E074E07FE08ADE
:106A9C00E095E0A0E0ABE0B6E0C1E0CCE0D7E0E20E
:106AAC00E0EDE0F8E103E10EE119E125E130E13B35
:106ABC00E146E151E15CE167E172E17DE188E1935E
:106ACC00E19EE1A9E1B4E1BFE1CAE1D5E1E0E1EB8E
:106ADC00E1F6E201E20CE217E222E22DE238E243B7
:106AEC00E24EE259E264E26FE27AE286E291E29CE3
:106AFC00E2A7E2B2E2BDE2C8E2D3E2DEE2E9E2F40E
:106B0C00E2FFE30AE315E320E32BE336E341E34C36
:106B1C00E357E362E36DE378E383E38EE399E3A465
:106B2C00E3AFE3BAE3C5E3D0E3DBE3E6E3F2E3FD93
:106B3C00E408E413E41EE429E434E43FE44AE455B5
:106B4C00E460E46BE476E481E48CE497E4A2E4ADE5
:106B5C00E4B8E4C3E4CEE4D9E4E4E4EFE4FAE50514
:106B6C00E510E51BE526E531E53CE547E552E55E3C
:106B7C00E569E574E57FE58AE595E5A0E5ABE5B665
:106B8C00E5C1E5CCE5D7E5E2E5EDE5F8E603E60E93
:106B9C00E619E624E62FE63AE645E650E65BE666BD
:106BAC00E671E67CE687E692E69DE6A8E6B3E6BFEC
:106BBC00E6CAE6D5E6E0E6EBE6F6E701E70CE71712
:106BCC00E722E72DE738E743E74EE759E764E76F3D
:106BDC00E77AE785E790E79BE7A6E7B1E7BCE7C76D
:106BEC00E7D2E7DDE7E8E7F3E7FEE809E814E81F9A
:106BFC00E82BE836E841E84CE857E862E86DE878BD
:106C0C00E883E88EE899E8A4E8AFE8BAE8C5E8D0EC
:106C1C00E8DBE8E6E8F1E8FCE907E912E91DE92818
:106C2C00E933E93EE949E954E95FE96AE975E98044
:106C3C00E98CE997E9A2E9ADE9B8E9C3E9CEE9D96C
:106C4C00E9E4E9EFE9FAEA05EA10EA1BEA26EA3197
:106C5C00EA3CEA47EA52EA5DEA68EA73EA7EEA89C4
:106C6C00EA94EA9FEAAAEAB5EAC0EACBEAD6EAE1F4
:106C7C00EAECEAF8EB03EB0EEB19EB24EB2FEB3A17
:106C8C00EB45EB50EB5BEB66EB71EB7CEB87EB9244
:106C9C00EB9DEBA8EBB3EBBEEBC9EBD4EBDFEBEA74
:106CAC00EBF5EC00EC0BEC16EC21EC2CEC37EC429D
:106CBC00EC4DEC59EC64EC6FEC7AEC85EC90EC9BC5
:106CCC00ECA6ECB1ECBCECC7ECD2ECDDECE8ECF3F4
:106CDC00ECFEED09ED14ED1FED2AED35ED40ED4B1D
:106CEC00ED56ED61ED6CED77ED82ED8DED98EDA34C
:106CFC00EDAEEDB9EDC5EDD0EDDBEDE6EDF1EDFC76
:106D0C00EE07EE12EE1DEE28EE33EE3EEE49EE549B
:106D1C00EE5FEE6AEE75EE80EE8BEE96EEA1EEACCB
:106D2C00EEB7EEC2EECDEED8EEE3EEEEEEF9EF04FA
:106D3C00EF0FEF1AEF25EF31EF3CEF47EF52EF5D1E
:106D4C00EF68EF73EF7EEF89EF94EF9FEFAAEFB54B
:106D5C00EFC0EFCBEFD6EFE1EFECEFF7F002F00D79
:106D6C00F018F023F02EF039F044F04FF05AF065A3
:106D7C00F070F07BF086F092F09DF0A8F0B3F0BECE
:106D8C00F0C9F0D4F0DFF0EAF0F5F100F10BF116F8
:106D9C00F121F12CF137F142F14DF158F163F16E23
:106DAC00F179F184F18FF19AF1A5F1B0F1BBF1C653
:106DBC00F1D1F1DCF1E7F1F2F1FEF209F214F21F7C
:106DCC00F22AF235F240F24BF256F261F26CF277A3
:106DDC00F282F28DF298F2A3F2AEF2B9F2C4F2CFD3
:106DEC00F2DAF2E5F2F0F2FBF306F311F31CF327FF
:106DFC00F332F33DF348F353F35FF36AF375F38027
:106E0C00F38BF396F3A1F3ACF3B7F3C2F3CDF3D852
:106E1C00F3E3F3EEF3F9F404F40FF41AF425F4307D
:106E2C00F43BF446F451F45CF467F472F47DF488AA
:106E3C00F493F49EF4A9F4B4F4BFF4CBF4D6F4E1D7
:106E4C00F4ECF4F7F502F50DF518F523F52EF539FC
:106E5C00F544F54FF55AF565F570F57BF586F5912A
:106E6C00F59CF5A7F5B2F5BDF5C8F5D3F5DEF5E95A
:106E7C00F5F4F5FFF60AF615F620F62BF637F64282
:106E8C00F64DF658F663F66EF679F684F68FF69AAA
:106E9C00F6A5F6B0F6BBF6C6F6D1F6DCF6E7F6F2DA
:106EAC00F6FDF708F713F71EF729F734F73FF74A03
:106EBC00F755F760F76BF776F781F78CF798F7A330
:106ECC00F7AEF7B9F7C4F7CFF7DAF7E5F7F0F7FB5A
:106EDC00F806F811F81CF827F832F83DF848F85382
:106EEC00F85EF869F874F87FF88AF895F8A0F8ABB2
:106EFC00F8B6F8C1F8CCF8D7F8E2F8EDF8F8F904E0
:106F0C00F90FF91AF925F930F93BF946F951F95C01
:106F1C00F967F972F97DF988F993F99EF9A9F9B431
:106F2C00F9BFF9CAF9D5F9E0F9EBF9F6FA01FA0C5F
:106F3C00FA17FA22FA2DFA38FA43FA4EFA59FA6588
:106F4C00FA70FA7BFA86FA91FA9CFAA7FAB2FABDB1
:106F5C00FAC8FAD3FADEFAE9FAF4FAFFFB0AFB15DF
:106F6C00FB20FB2BFB36FB41FB4CFB57FB62FB6D09
:106F7C00FB78FB83FB8EFB99FBA4FBAFFBBAFBC539
:106F8C00FBD1FBDCFBE7FBF2FBFDFC08FC13FC1E5E
:106F9C00FC29FC34FC3FFC4AFC55FC60FC6BFC7689
:106FAC00FC81FC8CFC97FCA2FCADFCB8FCC3FCCEB9
:106FBC00FCD9FCE4FCEFFCFAFD05FD10FD1BFD26E5
:106FCC00FD32FD3DFD48FD53FD5EFD69FD74FD7F09
:106FDC00FD8AFD95FDA0FDABFDB6FDC1FDCCFDD739
:106FEC00FDE2FDEDFDF8FE03FE0EFE19FE24FE2F64
:106FFC00FE3AFE45FE50FE5BFE66FE71FE7CFE8791
:10700C00FE92FE9EFEA9FEB4FEBFFECAFED5FEE0B9
:10701C00FEEBFEF6FF01FF0CFF17FF22FF2DFF38E2
:10702C00FF43FF4EFF59FF64FF6FFF7AFF85FF9010
:10703C00FF9BFFA6FFB1FFBCFFC7FFD2FFDDFFE840
:0C704C00FFF3FFFE3031323334353637AD
:10409A00C100C10141004700C10241004800680057
:1040AA000063000000010001000200020003000496
:1040BA0000040005000500060006000700080008C5
:1040CA0000090009000A000B000B000C000C000D8F
:1040DA00000D000E000F000F00100010001100125A
:1040EA000012001300130014001500150016001624
:1040FA0000170017001800190019001A001A001BEF
:10410A00001C001C001D001D001E001E001F0020B8
:10411A000020002100210022002300230024002483
:10412A00002500260026002700270028002800294D
:10413A00002A002A002B002B002C002D002D002E17
:10414A00002E002F002F00300031003100320032E3
:10415A0000330034003400350035003600360037AD
:10416A000038003800390039003A003B003B003C77
:10417A00003C003D003E003E003F003F0040004042
:10418A00004100420042004300430044004500450C
:10419A000046004600470047004800490049004AD7
:1041AA00004A004B004C004C004D004D004E004FA1
:1041BA00004F00500050005100510052005300536C
:1041CA000054005400550056005600570057005836
:1041DA0000580059005A005A005B005B005C005D01
:1041EA00005D005E005E005F0060006000610061CB
:1041FA000062006200630064006400650065006696
:10420A00006700670068006800690069006A006B5F
:10421A00006B006C006C006D006E006E006F006F2A
:10422A0000700071007100720072007300730074F4
:10423A0000750075007600760077007800780079BE
:10424A000079007A007A007B007C007C007D007D8A
:10425A00007E007F007F0080008000810081008254
:10426A00008300830084008400850086008600871E
:10427A000087008800890089008A008A008B008BE9
:10428A00008C008D008D008E008E008F00900090B3
:10429A00009100910092009200930094009400957E
:1042AA000095009600970097009800980099009A48
:1042BA00009A009B009B009C009C009D009E009E13
:1042CA00009F009F00A000A100A100A200A200A3DD
:1042DA0000A300A400A500A500A600A600A700A8A8
:1042EA0000A800A900A900AA00AB00AB00AC00AC72
:1042FA0000AD00AD00AE00AF00AF00B000B000B13D
:10430A0000B200B200B300B300B400B400B500B606
:10431A0000B600B700B700B800B900B900BA00BAD1
:10432A0000BB00BC00BC00BD00BD00BE00BE00BF9B
:10433A0000C000C000C100C100C200C300C300C465
:10434A0000C400C500C500C600C700C700C800C831
:10435A0000C900CA00CA00CB00CB00CC00CC00CDFB
:10436A0000CE00CE00CF00CF00D000D100D100D2C5
:10437A0000D200D300D400D400D500D500D600D690
:10438A0000D700D800D800D900D900DA00DB00DB5A
:10439A0000DC00DC00DD00DD00DE00DF00DF00E025
:1043AA0000E000E100E200E200E300E300E400E5EF
:1043BA0000E500E600E600E700E700E800E900E9BA
:1043CA0000EA00EA00EB00EC00EC00ED00ED00EE84
:1043DA0000EE00EF00F000F000F100F100F200F34F
:1043EA0000F300F400F400F500F600F600F700F719
:1043FA0000F800F800F900FA00FA00FB00FB00FCE4
:10440A0000FD00FD00FE00FE00FF00FF01000101AB
:10441A000101010201020103010401040105010570
:10442A000106010701070108010801090109010A3A
:10443A00010B010B010C010C010D010E010E010F04
:10444A00010F0110011001110112011201130113D0
:10445A00011401150115011601160117011701189A
:10446A0001190119011A011A011B011C011C011D64
:10447A00011D011E011F011F01200120012101212F
:10448A0001220123012301240124012501260126F9
:10449A0001270127012801280129012A012A012BC4
:1044AA00012B012C012D012E013001310132013382
:1044BA0001340135013701380139013A013B013C28
:1044CA00013E013F014001410142014301450146CC
:1044DA00014701480149014A014C014D014E014F72
:1044EA000150015201530154015501560157015916
:1044FA00015A015B015C015D015E016001610162BB
:10450A00016301640165016701680169016A016B60
:10451A00016C016E016F0170017101720173017505
:10452A000176017701780179017B017C017D017EA9
:10453A00017F01800182018301840185018601874F
:10454A000189018A018B018C018D018E01900191F3
:10455A000192019301940195019701980199019A99
:10456A00019B019D019E019F01A001A101A201A43D
:10457A0001A501A601A701A801A901AB01AC01ADE2
:10458A0001AE01AF01B001B201B301B401B501B688
:10459A0001B701B901BA01BB01BC01BD01BE01C02D
:1045AA0001C101C201C301C401C601C701C801C9D1
:1045BA0001CA01CB01CD01CE01CF01D001D101D277
:1045CA0001D401D501D601D701D801D901DB01DC1B
:1045DA0001DD01DE01DF01E001E201E301E401E5C1
:1045EA0001E601E801E901EA01EB01EC01ED01EF65
:1045FA0001F001F101F201F301F401F601F701F80A
:10460A0001F901FA01FB01FD01FE01FF02000201AD
:10461A000202020402050206020702080209020B4C
:10462A00020C020D020E020F0211021202130214F0
:10463A000215021602180219021A021B021C021D96
:10464A00021F02200221022202230224022602273A
:10465A0002280229022A022B022D022E022F0230E0
:10466A000231023302340235023602370238023A84
:10467A00023B023C023D023E023F02410242024329
:10468A0002440245024602480249024A024B024CCF
:10469A00024D024F02500251025202530254025674
:1046AA000257025A025C025F0261026302660268F2
:1046BA00026A026D026F0272027402760279027B4A
:1046CA00027D02800282028402870289028B028EA4
:1046DA0002900292029502970299029C029E02A1FE
:1046EA0002A302A502A802AA02AC02AF02B102B357
:1046FA0002B602B802BA02BD02BF02C102C402C6B1
:10470A0002C902CB02CD02D002D202D402D702D908
:10471A0002DB02DE02E002E202E502E702E902EC63
:10472A0002EE02F102F302F502F802FA02FC02FFBB
:10473A000301030303060308030A030D030F03110E
:10474A00031403160318031B031D03200322032467
:10475A0003270329032B032E0330033203350337C0
:10476A000339033C033E0340034303450348034A1A
:10477A00034C034F0351035303560358035A035D73
:10478A00035F0361036403660368036B036D036FCE
:10479A000372037403770379037B037E0380038226
:1047AA0003850387038C03900395039A039F03A34E
:1047BA0003A803AD03B103B603BB03BF03C403C914
:1047CA0003CE03D203D703DC03E003E503EA03EED7
:1047DA0003F303F803FD04010406040B040F041495
:1047EA000419041E04220427042C04300435043A54
:1047FA00043E04430448044D04510456045B045F18
:10480A0004640469046D04720477047C04800485DA
:10481A00048A048E04930498049C04A104A604AB9D
:10482A0004AF04B404BD04C704D004DA04E304ECFE
:10483A0004F604FF05090512051B0525052E053892
:10484A000541054B0554055D05670570057A058325
:10485A00058C0596059F05A905B205BB05C505CEBC
:10486A0005D805E10734088609D90B2B0C7E0DD033
:10487A000F23107511C8131A146D15C01712186575
:10488A0019B71B0A1C5C1DAF1F01205421A722F96E
:10489A00244C259E26F1284329962AE82C3B2D8D67
:1048AA002EE041086300410864004108650042089F
:1048BA0066000041086800420869000041000000E3
:1048CA004100010141086B0042000200004200045D
:1048DA0000004200060000420008000042000A00F0
:1048EA000042000C000041086C0041086D8041083C
:0748FA006E8042086F000010
:10940500E4F584758810758902758E02758A017573
:069415008C0143A80222B5
:0D941B00E4F584759A4075F809759D3022BE
:1092C300E4F58475E880900863E0F5BB7584027566
:1092D300BCF975E880A3E0F5BBE4F58443E712220B
:074FFF00E4F58475D10222E4
:10938C0075840FE4F5AD75A4CF75A50175A67F7531
:09939C00A77F75E10375E340228F
:108F9500E4FFFE75840F438A0353A1DFF58475B79B
:108FA5003075840F43A120438901758D01758F01AB
:108FB500758E040FBF00010EEF640F4E70F54389E7
:108FC50002E58920E4130FBF00010EBE0FF3BFFFBA
:0C8FD500F0E4F58443EF1080E87597028B
:018FE100226D
:10930200128F9512938C12940512941B124FFF1216
:0E93120092C3900046E0FF12942843F6022218
:06503300E4900865F02284
:079466009008657401F0227B
:107FE5007B017A0D793B12919AEF70030281E09043
:107FF5000D3DE024FC606A1470030280AE24F1603C
:108005002924FD601D24FD602624FD604814604B75
:10801500240860030280FF9000477401F0C2090242
:1080250080FFE4900047F00280FFD2020280FF7BD0
:10803500017A0D793B900D4BEBF0A3EAF0A3E9F043
:10804500124A4CFE900046E0FF6E60030280FF126C
:1080550092A20280FF1294660280FF1250330280C2
:10806500FF7B017A0D793B900D4EEBF0A3EAF0A36F
:10807500E9F0900003124A65FF900046E06F707AC0
:10808500A3E0606E900D4EEBF0A3EAF0A3E9F0904B
:108095000005124A65FF900006124A65FD9000042E
:1080A500124A65FB128B6680497B017A0D793B90FC
:1080B5000D4EEBF0A3EAF0A3E9F0900003124A6538
:1080C500FF900046E06F7032A3E06026900D4EEB06
:1080D500F0A3EAF0A3E9F0900005124A65FF9000CD
:1080E50006124A65FD900004124A65FB128AB01219
:1080F50091C6900046E0FF1292E3900047E07003BE
:10810500027FE5900D3DE014603524FA605414704B
:10811500030281AE24066003027FE512501B7B013A
:108125007A0D793B900D4BEBF0A3EAF0A3E9F090C3
:108135000003124A65900D0AF012947F0281DA124B
:10814500501B7B017A0D793B900D4BEBF0A3EAF0C8
:10815500A3E9F0900003124A65900D0AF01291C64A
:10816500807312501B7B017A0D793B900D51EBF01A
:10817500A3EAF0A3E9F0900003124A65FF9000041A
:10818500124A65FD900005124A65FBC003900D512A
:10819500E0FBA3E0FAA3E0F9900006124A65900D12
:1081A50077F0D0031289E5802C12501B7B017A0DE4
:1081B500793B900D51EBF0A3EAF0A3E9F0900003B1
:1081C500124A65FF900004124A65FD900005124AA7
:0B81D50065FB1281E1129435027FE58A
:0181E000227C
:104FA80075FFDE75FFAD9000467460F0129302D273
:104FB800AF1293D61291C6AF84E4F5848F84900023
:104FC80048E0600812947FE4900048F030001090A8
:104FD8000046E0FF7BFF7A50793C128EE6C2003033
:104FE8000110900865E07008900046E0FF12928179
:074FF800C201127FE580C039
:03500600027058DD
:10705800C0E0C0F0C083C082C0D075D000C000C0FE
:0D70680001C002C003C004C005C006C0077F
:1070750090086AE004F07006900869E004F0C39097
:10708500086AE09404900869E0940050030278339C
:10709500900869E4F0A3F0900CD9740FF0A374FF85
:1070A500F0A37408F0A37420F0900868E014600F52
:1070B5001460111460392403703812502C80331277
:1070C5009455802E900866E4F0A3F0127BA99008F1
:1070D50067E004F07006900866E004F0C390086766
:1070E500E09408900866E06480948040DE80031296
:1070F500933D900868E004F0C3648094844002E402
:10710500F0900CDBE0FEA3E0FF900CD9E0FCA3E0DF
:10711500FD124CCA900CD5124C36900868E0FF75EC
:0D712500F002124A2AAFF0EF700302783337
:07713200900CDFE4F0A3F074
:10713900900CE0E025E0FF900CDFE033FE74442F73
:10714900F974503EFA900CFD74FFF0A3EAF0A3E93C
:10715900F0900CFDE0FBA3E0FAA3E0F9124A4CFD24
:10716900540FFB900D00E4F0A3EBF0EDC4540FFDB8
:10717900A3E4F0A3EDF0900CFDE0FB900001124AAE
:1071890065540FFD900D04E4F0A3EDF0740B2FF599
:1071990082740D3EF583E0FEA3E0FFE4FCFD900D53
:1071A90006124C36900CDFE0FEA3E0FF4E6006EFBE
:1071B90064054E7016900D01E025E0FF900D00E08A
:1071C90033FE74262FF58274008014900CE0E025BC
:1071D900E0FF900CDFE033FE74152FF582740D3E4D
:1071E900F583E0FEA3E0FFE4FCFD900CF5124C36BC
:1071F900900CF5E0F8A3E0F9A3E0FAA3E0FBC3746F
:10720900FF9BFF740F9AFEE499FDE498FCA3124CCE
:1072190036900D06E0FCA3E0FDA3E0FEA3E0FFE449
:10722900FBFAF9F8D3124C255069E47FAA7E02FDD6
:10723900FC900D06E0F8A3E0F9A3E0FAA3E0FBC394
:10724900124C25504E7F607EF07DFF7CFF900D062D
:10725900E0F8A3A3A3E0124AF2900CE5124C369091
:107269000CE5E0FCA3E0FDA3E0FEA3E0FFE47BAABC
:107279007A02F9F81290B1900CE5124C36900CE5AF
:10728900E0FCA3E0FDA3E0FEA3E02428FFEE342305
:1072990002731C900D06E0FCA3E0FDA3E0FEA3E051
:1072A900FFE47BAA7A02F9F8D3124C255072E4FF65
:1072B9007E10FDFC900D06E0F8A3E0F9A3E0FAA327
:1072C900E0FBC3124C2550587F787EEC7DFF7CFF94
:1072D900900D06E0F8A3A3A3E0124AF2900CE51280
:1072E9004C36900CE5E0FCA3E0FDA3E0FEA3E0FF33
:1072F900E47B567A0DF9F81290B1900CE5124C36F0
:10730900900CE5E0FCA3E0FDA3E0FEA3E0246FFF01
:10731900EE3417FEE43DFDE43CFC900CE5124C36DE
:10732900900CE5E0FCA3E0FDA3E0FEA3E0FF900CD8
:10733900ED124C36900CE5E0FCA3E0FDA3E0FEA3C2
:10734900E0FF900CF1124C36900CF5E0FCA3E0FD47
:10735900A3E0FEA3E0FF900CE1124C36900CE1E0B3
:10736900FCA3E0FDA3E0FEA3E0FFE4FBFAF9F8D3F8
:10737900124C0F504DE4FF7E08FDFC900CE1E0F843
:10738900A3E0F9A3E0FAA3E0FBC3124C0F5033E4E6
:107399007FF47E01FDFC900CE1E0F8A3A3A3E012C9
:1073A9004AF2900CE5124C36900CE5E0FCA3E0FDA6
:1073B900A3E0FEA3E0FFE4FB7A08F9F81290B1021A
:1073C90074DB900CE1E0FCA3E0FDA3E0FEA3E0FF89
:1073D900E4FB7A08F9F8D3124C0F506FE4FF7E0CE6
:1073E900FDFC900CE1E0F8A3E0F9A3E0FAA3E0FBCF
:1073F900C3124C0F5055E47FDC7E05FDFC900CE177
:10740900E0F8A3A3A3E0124AF2900CE5124C3690DF
:107419000CE5E0FCA3E0FDA3E0FEA3E0FFE4FB7ABA
:1074290004F9F81290B1900CE5124C36900CE5E095
:10743900FCA3E0FDA3E0FEA3E0243CFFEE34F6FE4E
:10744900ED34FFFDEC34FFFC0274DB900CE1E0FC51
:10745900A3E0FDA3E0FEA3E0FFE4FB7A0CF9F8D377
:10746900124C0F5073E4FF7E10FDFC900CE1E0F824
:10747900A3E0F9A3E0FAA3E0FBC3124C0F5059E4CF
:107489007F587E1BFDFC900CE1E0F8A3A3A3E0125A
:107499004AF2900CE5124C36900CE5E0FCA3E0FDB5
:1074A900A3E0FEA3E0FFE47BFF7A03F9F81290B1B1
:1074B900900CE5124C36900CE5E0FCA3E0FDA3E04E
:1074C900FEA3E024B3FFEE34B5FEED34FFFDEC344A
:1074D900FFFC900CE5124C36900CEDE0F8A3E0F9B6
:1074E900A3E0FAA3E0FB900CE5E0FCA3E0FDA3E038
:1074F900FEA3E0FFEB2FFFEA3EFEE93DFDE83CFC81
:10750900900CED124C36900CF9E0FCA3E0FDA3E0E1
:10751900FEA3E0FF900CE1124C36900CE1E0FCA3D5
:10752900E0FDA3E0FEA3E0FFE4FBFAF9F8D3124C77
:107539000F504DE4FF7E08FDFC900CE1E0F8A3E05C
:10754900F9A3E0FAA3E0FBC3124C0F5033E47FF434
:107559007E01FDFC900CE1E0F8A3A3A3E0124AF23E
:10756900900CE5124C36900CE5E0FCA3E0FDA3E09D
:10757900FEA3E0FFE4FB7A08F9F81290B1027699CC
:10758900900CE1E0FCA3E0FDA3E0FEA3E0FFE4FB37
:107599007A08F9F8D3124C0F506FE4FF7E0CFDFC0A
:1075A900900CE1E0F8A3E0F9A3E0FAA3E0FBC31231
:1075B9004C0F5055E47FDC7E05FDFC900CE1E0F8B2
:1075C900A3A3A3E0124AF2900CE5124C36900CE505
:1075D900E0FCA3E0FDA3E0FEA3E0FFE4FB7A04F9ED
:1075E900F81290B1900CE5124C36900CE5E0FCA332
:1075F900E0FDA3E0FEA3E0243CFFEE34F6FEED340B
:10760900FFFDEC34FFFC027699900CE1E0FCA3E06D
:10761900FDA3E0FEA3E0FFE4FB7A0CF9F8D3124CDA
:107629000F5073E4FF7E10FDFC900CE1E0F8A3E03D
:10763900F9A3E0FAA3E0FBC3124C0F5059E47F58B9
:107649007E1BFDFC900CE1E0F8A3A3A3E0124AF233
:10765900900CE5124C36900CE5E0FCA3E0FDA3E0AC
:10766900FEA3E0FFE47BFF7A03F9F81290B1900CD6
:10767900E5124C36900CE5E0FCA3E0FDA3E0FEA387
:10768900E024B3FFEE34B5FEED34FFFDEC34FFFC2E
:10769900900CE5124C36900CF1E0F8A3E0F9A3E068
:1076A900FAA3E0FB900CE5E0FCA3E0FDA3E0FEA358
:1076B900E0FFEB2FFFEA3EFEE93DFDE83CFC900CC4
:1076C900F1124C36E47F167E03FDFC900CEDE0F8D8
:1076D900A3E0F9A3E0FAA3E0FB124AF2900CE91245
:1076E9004C36900CE9E0FCA3E0FDA3E0FEA3E0FF2B
:1076F900E47B64FAF9F8124B7D900CE9124C36E4FC
:107709007FFF7EFFFDFC900CE9E0F8A3E0F9A3E020
:10771900FAA3E0FBD3124C25400A900CE9124C4223
:107729000000FFFF900CE9A3A3E0FEA3E0FDAC0677
:10773900900D03E025E0FF900D02E033FE744B2F1E
:10774900F58274003EF583ECF0A3EDF0E47F167E3C
:1077590003FDFC900CF1E0F8A3E0F9A3E0FAA3E043
:10776900FB124AF2900CE9124C36900CE9E0FCA3AA
:10777900E0FDA3E0FEA3E0FFE47B64FAF9F8124B15
:107789007D900CE9124C36E47FFF7EFFFDFC900CE6
:10779900E9E0F8A3E0F9A3E0FAA3E0FBD3124C2552
:1077A900400A900CE9124C420000FFFF900CE9A33B
:1077B900A3E0FEA3E0FDAC06900D05E025E0FF90F7
:1077C9000D04E033FE744B2FF58274003EF583EC13
:0477D900F0A3EDF03C
:1077DD00900CE0E004F07006900CDFE004F0900CEB
:1077ED00DFE07004A3E06406600302713978DD7C8C
:1077FD000C7D017B017A00795F7E007F02124A04C5
:10780D00785F7C007D017B017A0079617E007F02CB
:10781D00124A0478617C007D017B017A0C79DD7E52
:06782D00007F02124A0474
:10783300D007D006D005D004D003D002D001D000A9
:0B784300D0D0D082D083D0F0D0E03253
:04502C0043E8102223
:09945500758402D2ECE4F58422D6
:107BA900900866E0FEA3E0FFEE6003027D0AEFB4F1
:107BB90008004003027D0A907BC7F8282873027BDE
:107BC900DF027C0B027C37027C63027C8E027CAC78
:107BD900027CCA027CE878ED7C0D7D017B017A008C
:107BE900795B7E007F02124A0478EF7C0D7D017B70
:107BF900017A00794B7E007F02124A04907050028C
:107C09007D0478ED7C0D7D017B017A00795D7E0034
:107C19007F02124A0478EF7C0D7D017B017A00799D
:107C29004D7E007F02124A04907051027D0478ED66
:107C39007C0D7D017B017A00795F7E007F02124A0B
:107C49000478EF7C0D7D017B017A00794F7E007FFE
:107C590002124A04907052027D0478ED7C0D7D0178
:107C69007B017A0079617E007F02124A0478EF7CF9
:107C79000D7D017B017A0079517E007F02124A0451
:107C89009070538076E4900DEDF0A3F078EF7C0DC1
:107C99007D017B017A007953FE7F02124A049070BC
:107CA900548058E4900DEDF0A3F078EF7C0D7D0140
:107CB9007B017A007955FE7F02124A049070558043
:107CC9003AE4900DEDF0A3F078EF7C0D7D017B0196
:107CD9007A007957FE7F02124A04907056801CE49C
:107CE900900DEDF0A3F078EF7C0D7D017B017A001A
:107CF9007959FE7F02124A04907057E493900DEC73
:107D0900F0E4F584C2FA900000E0F59B30FFFDC273
:107D1900FFE4FFFE0FBF00010EEF64324E70F590D5
:107D29000DECE0F59B30FFFDC2FFE4FEFF0FBF0045
:107D3900010EEF64324E70F5900DEDE0F59B30FFCA
:107D4900FDC2FFE4FEFF0FBF00010EEF64324E706B
:107D5900F5900DEEE0F59B30FFFDC2FFE4FEFF0F4D
:107D6900BF00010EEF64324E70F5900000E0F59B04
:107D790030FFFDC2FFE4FEFF0FBF00010EEF6432CA
:107D89004E70F5900DECE0F59B30FFFDC2FFE4FE6F
:107D9900FF0FBF00010EEF64324E70F5900DEFE05A
:107DA900F59B30FFFDC2FFE4FEFF0FBF00010EEFA0
:107DB90064324E70F5900DF0E0F59B30FFFDC2FF87
:107DC900E4FEFF0FBF00010EEF64324E70F5D2FAE8
:017DD9002287
:03503000027DDA24
:107DDA00C0E0C0F0C083C082C0D075D000C000C06F
:0D7DEA0001C002C003C004C005C006C007F0
:107DF70053E8DFAFBFEFFEADBE7C00E42DFFEC3EE6
:107E0700900023F0A3EFF0900023E0FCA3E0FD90A7
:107E17000863E0FF3395E0FEEF25E0FFEE33FE74E5
:107E2700262FF58274003EF583ECF0A3EDF0900861
:107E370063E004F0C3648094885003027FC4E4F0D5
:107E4700900030E0FFA3E090000FCFF0A3EFF09099
:107E5700002EE0FFA3E0900011CFF0A3EFF0900019
:107E67002CE0FFA3E0900013CFF0A3EFF090002ADF
:107E7700E0FFA3E0900015CFF0A3EFF0900028E01B
:107E8700FFA3E0900017CFF0A3EFF0900026E0FFEC
:107E9700A3E0900019CFF0A3EFF090003EE0FFA31E
:107EA700E090001BCFF0A3EFF0900040E0FFA3E0CD
:107EB70090001DCFF0A3EFF0900042E0FFA3E09009
:107EC700001FCFF0A3EFF0900044E0FFA3E0900085
:107ED70021CFF0A3EFF0900001E06037E4FFEF253A
:107EE700E0240FF582E43400F583E0FCA3E0FDEF26
:107EF70025E02454F582E4340DF583ECF0A3EDF08E
:107F07000FEFB40AD9900001E004F0E0D3940F40DA
:107F170002E4F0900001E070047D0180027D007FA3
:107F27000012784E900001E070047D0180027D0010
:107F37007F0112784E900001E070047D0180027D80
:107F4700007F0212784E900001E070047D018002EC
:107F57007D007F0312784E900001E070047D018060
:107F6700027D007F0412784E900001E070047D01CD
:107F770080027D007F0512784E900001E070047D3D
:107F87000180027D007F0612784E900001E07004A8
:107F97007D0180027D007F0712784E900001E0701E
:107FA700047D0180027D007F0812784E900001E079
:107FB70070047D0180027D007F0912784E9008636E
:037FC700E0F5BB27
:107FCA00D007D006D005D004D003D002D001D0000B
:0B7FDA00D0D0D082D083D0F0D0E032B5
:03503900028E18CC
:108E1800C0E0C0F0C083C082C0D075D000C005C01B
:108E280006C007758402C2ED900025E5BEF0E07526
:108E3800F010A4FD900864E0FF3395E0FEEF25E014
:108E4800FFEE33FE74362FF58274003EF583E5F0AD
:108E5800F0A3EDF0900864E004F0C36480948840C7
:108E680002E4F0900864E0F5BB758400D007D006F2
:0D8E7800D005D0D0D082D083D0F0D0E03231
:104D230090003AE0FFA3E0900002CFF0A3EFF090F1
:104D3300003CE0FEA3E0FF900004EEF0A3EFF0D30D
:104D4300900007E09F900006E09E5016900004E05C
:104D5300FFA3E0A3CFF0A3EFF090000AE4F0A37465
:104D630080F0900008E0FEA3E0FF900002E0FCA3C7
:104D7300E0FDC39FEC9E4011900008ECF0A3EDF022
:104D830090000CE4F0A37480F0900047E024FF92BD
:104D930087900004E0FEA3E0FFD394A3EE940040C9
:104DA30003D38001C392B0D3EF94F4EE9400400395
:104DB300D38001C392B1900004E0FEA3E0FFD3943B
:104DC3003BEE94024003D38001C392B2D3EF94D35A
:104DD300EE94034003D38001C392B3900004E0FE3A
:104DE300A3E0FFD394BCEE94054003D38001C392A8
:104DF300B4D3EF9433EE940A4003D38001C392B546
:104E0300D3900005E0944C900004E0940F4003D34A
:104E13008001C392B6D390000BE0940090000AE0A7
:104E230094004070900006E0FEA3E0FFD3944CEEA4
:104E3300940F4004D2B6804CD3EF9433EE940A40DF
:104E430004D2B5803FD3EF94BCEE94054004D2B4B2
:104E53008032D3EF94D3EE94034004D2B38025D3AE
:104E6300EF943BEE94024004D2B28018D3EF94F453
:104E7300EE94004004D2B1800BD3EF94A3EE9400E0
:104E83004002D2B090000BE024FFF090000AE0341F
:104E9300FFF08007E4900006F0A3F0900002E0FE2C
:104EA300A3E0FFD394A3EE94004003D38001C39205
:104EB300A0D3EF94F4EE94004003D38001C392A1F6
:104EC300900002E0FEA3E0FFD3943BEE9402400384
:104ED300D38001C392A2D3EF94D3EE94034003D3C0
:104EE3008001C392A3900002E0FEA3E0FFD394BC31
:104EF300EE94054003D38001C392A4D3EF9433EE21
:104F0300940A4003D38001C392A5D3900003E09495
:104F13004C900002E0940F4003D38001C392A6D3C8
:104F230090000DE0940090000CE09400406F90001E
:104F330008E0FEA3E0FFD3944CEE940F4004D2A606
:104F4300804CD3EF9433EE940A4004D2A5803FD330
:104F5300EF94BCEE94054004D2A48032D3EF94D3F3
:104F6300EE94034004D2A38025D3EF943BEE940246
:104F73004004D2A28018D3EF94F4EE94004004D2FC
:104F8300A1800BD3EF94A3EE94004002D2A0900033
:104F93000DE024FFF090000CE034FFF022E49000D9
:044FA30008F0A3F07F
:014FA70022E7
:108D190090086DE0A3F0E5B0548090086DF0A3E0F1
:108D2900FD90086DE0FE6D90000EF0EE7032ED6082
:108D390007E490086FF0A3F0900870E004F0700663
:108D490090086FE004F0D3900870E0948090086F69
:108D5900E09401404090086CE0703AD20004F0229F
:108D690090086EE0702FC3900870E094D090086F5F
:108D7900E09400501B300209900047E06401F08044
:108D89000F900047E06009A37401F0E4900047F0F8
:058D9900E490086CF0FD
:018D9E0022B2
:10933D0090086BE0FF7005128D198007EFB40103E3
:0B934D00124D2390086BE06401F02239
:10906D00AB84A2AF9206E4FCFDED900DF1124C36EF
:10907D00900DF3E0FEA3E0780EA60608F6E4F58465
:10908D00C2AF43B701438F02438F0118E6FE08E6D6
:10909D00F5828E83E4F053B7FEF58FA20692AFAF43
:0390AD00038F84AA
:0190B000229D
:028F4600AB0579
:108F4800AA84A2AF9207E4FCFDED900DF5124C3611
:108F5800EBFF3395E0FEEFF44E6029900DF7E0FE4D
:108F6800A3E07810A60608F6E4F584C2AF43B7017B
:108F7800758F0118E6FC08E6F5828C83EBF053B791
:0C8F8800FEE4F58FA20792AFAF028F84C9
:018F940022BA
:108E8500900DDAEEF0A3EFF0A3ECF0A3EDF0A3EA7A
:108E9500F0A3EBF0900DDEE07002A3E06042900DD0
:108EA500DAE0FEA3E0FFA3E0FCA3E0F5828C83E01B
:108EB500FD128F46900DDFE024FFF0900DDEE034CB
:108EC500FFF0900DDDE004F07006900DDCE004F09D
:108ED500900DDBE004F070BC900DDAE004F080B496
:018EE500226A
:08945E00E4900C71F0A3F02270
:1091EF00900C71E0FEA3E0FF12906D900C71E0FE09
:1091FF00A3E0FF7C087D717B007A04128E85E490DA
:06920F000C71F0A3F02237
:0A8C8D00A905900DE0EEF0A3EFF052
:108C9700EE54FCFE900C71E0FCA3E0FD7002EE6C5C
:108CA7006057ED4C60031291EF900DE0E0FEEE543B
:108CB700FCFE7F00900C71F0A3EFF0900DE2EEF058
:108CC700A3EFF0A37408F0A37471F07E04900DE293
:108CD700E475F001124ADC85F082F583E493FD9098
:108CE7000DE4E475F001124ADC85F082F583EDF0BE
:108CF700EF1F70011EEF4E70D4900DE0E0FCA3E073
:108D0700FDEC5403FC74712DF58274083CF583E97E
:018D1700F06B
:018D18002238
:108FE200900DCCEEF0A3EFF0A3EBF0A3EAF0A3E92F
:108FF200F0900DD174FFF5F0124ADC45F060269036
:109002000DCCE475F001124ADCAFF0FE900DCEE01B
:10901200FBA3E475F001124ADCA9F0FA124A4CFDF6
:06902200128C8D80CC22AF
:10490100420C760000420C7B0000420C7D0000C18D
:0549110004C105C10313
:0A944B00C205C204E4900CBFF02239
:10921500E4900C76F0A3F0900C7BF0A3F0900C7F1B
:10922500F0900C7DF0A3F0900C79F0A37440F0E47D
:05923500900C78F0220E
:06946D0012944B0292155F
:1093A500E4F5848FC343C30175C04475CF8EC2C332
:0993B50043E602900C7404F0225E
:10501B00E4F58420C7FDC2C212946DE4900C74F0C9
:01502B002262
:0B943500E4F584D2C2900C7404F02215
:0D942800AE071293A5900C75EFF002946D45
:10923A00E4900E0CF0A3F0300502FF222004FDD2C8
:10924A0005900CC0E4F0A37410F0900CC3EFF0E4A6
:04925A00A3F07F01FD
:01925E0022ED
:1091660030050A900CC0E07002A3E070037F002275
:10917600900CC1E024FFF0900CC0E034FFF0900C9E
:10918600C4E0FE04F074C52EF582E4340CF583EFDA
:04919600F07F012243
:0B944000300507C205D20412500922BB
:0E500900AF84E4F58420C7FDC2C4D2C58F84F5
:015017002276
:108D9F00900DD4EBF0A3EAF0A3E9F0900C74E0701F
:108DAF0002FF22900DD7E0FE6005D3941040037FA1
:088DBF00002212923AEF604E0F
:108DC700E4900DD9F0900DD7E0FF900DD9E0FEC3E8
:108DD7009F5024900DD4E0FBA3E0FAA3E0F98E8224
:108DE700758300124A65FF129166EF7002FF2290A9
:108DF7000DD9E004F080CEE4900CBFF012944090BF
:0E8E07000DD8E070032004FD900CBFE0FF22A8
:038E15007FFF22BA
:0E87D300900DF9EBF0A3EAF0A3E9F0A3EDF0AE
:1087E100E4FFD3900C77E09400900C76E0648094E1
:1087F1008050012253E6FD900C7DE0FEA3E0247F32
:10880100F582740C3EF583E0FF900C7DE475F00178
:10881100124AC6FCE5F064404C7006900C7DF0A352
:10882100F0900C7AE004F07006900C79E004F0E42A
:10883100FE900DFCE0FDEEC39D5054EEC39F504FE2
:10884100900C7DE0FCA3E0247FF582740C3CF58361
:10885100E0FD900DF9E0FBA3E0FAA3E0F98E82754B
:108861008300ED124AA4900C7DE475F001124AC612
:10887100FCE5F064404C7006900C7DF0A3F0900C88
:108881007AE004F07006900C79E004F00E80A2EE1C
:10889100C39F5029900C7DE475F001124AC6FCE596
:1088A100F064404C7006900C7DF0A3F0900C7AE0DF
:1088B10004F07006900C79E004F00E80D2900C77F1
:1088C100E024FFF0900C76E034FFF043E602900DD7
:0C88D100FCE0FEEFC39E50028002AF06E8
:0188DD002278
:1093BE00D3900C77E09400900C76E064809480401B
:0893CE00047F0180027F0022F0
:0350180002867598
:10867500C0E0C0F0C083C082C0D075D000C000C0CB
:0386850006C00725
:10868800C208AFC1EF124C7386BE0886BE1086CEF4
:108698001886D32086E028870D3087183887206011
:1086A800871B68872070871B788728808728908792
:1086B8009FA0000087AD900CC3E0F5C2C2C5900C26
:1086C800C2E4F00287AF900CC48028900CBF74FD00
:1086D800F0D2C4D2C50287AF900CC4E0FF900CC2A0
:1086E800E0C39F5014E0FF04F074C52FF582E43412
:1086F8000CF583E0F5C20287AFD2C4900CBFE4F05A
:10870800C2040287AFD2C5900CBF74FEF00287AFD7
:108718000287A4D2030287AF900C73E4F00287AFFC
:10872800900C73E07020E5C2F0E0FFC3900C7AE093
:108738009F7480F8900C79E0648098500312921529
:10874800900C73E004F0900C7AE024FFF0900C7920
:10875800E034FFF0900C7BE0FEA3E0247FF5827408
:108768000C3EF583E5C2F0900C7BE475F001124AEB
:10877800C6FEE5F064404E7006900C7BF0A3F090C6
:108788000C73E014F07020900C77E004F0701890EF
:108798000C76E004F0801030030DC203900CC2E4A4
:1087A800F0D2C58002D20830080EC2C6D2C6C2C5F1
:0A87B800C2C4D2C2C208C204C2C388
:1087C200D007D006D000D0D0D082D083D0F0D0E075
:0187D2003274
:05947300A2C7E433FF75
:0194780022D1
:06947900C2C253E6FD2211
:1083A100900DAAE0FFA3E0FCA3E0FDA3E0FBA3E0A6
:1083B100FAA3E0F9900D6EE508F0E509A3F0900D40
:0683C100B2E0900D70F027
:1083C700900D68EFF0A3ECF0A3EDF0A3EBF0A3EAB8
:0483D700F0A3E9F036
:1083DB00900D717403F0A374E8F0A3E584F0E4F559
:1083EB008420C7FDC2C4D2C2D2C5E4FF900E11F0E7
:1083FB0030C3FDAEC1EE24F8602324F8601F24F8CF
:10840B00602F24F8603624F8603A24F87003028455
:10841B00B324F870030284BB24380284C3EF700CBE
:10842B00900D68E025E044A0F5C27F03C2C502842D
:10843B00C9900D69E0F5C27F050284C9900E1174D5
:10844B0003F0807AEFB4050B900D69A3E0F5C27FC2
:10845B0006806BEF6406703E900D70E0900D6B70B4
:10846B000FE0FBA3E475F001124ADCA9F0FA8008D7
:10847B00E0FBA3E0FAA3E0F9124A4CF5C2900D6FB2
:10848B00E024FFF0900D6EE034FFF0E07002A3E00B
:10849B00702C7F078028EFB40706D2C47F09801E9B
:1084AB00900E117405F08016900E117404F0800E6E
:1084BB00900E117406F08006900E117401F0EFB45B
:1084CB000904C2C38036900E11E0B4031C900D71E9
:1084DB0074FFF5F0124AC645F0600ED2C4D2C5D275
:1084EB00C2C2C3E4900E11F0FF900E11E06008C2FF
:1084FB00C5D2C4C2C38005C2C30283FB20C7FD9093
:05850B000D73E0F58492
:018510002248
:10851100900D80EFF0A3ECF0A3EDF0A3EBF0A3EA54
:04852100F0A3E9F0EA
:10852500900D887403F0A374E8F0A3E584F0E4F5F6
:108535008420C7FDD2C2C2C4D2C5E4FF900E11F09B
:1085450030C3FDAEC1EE124C738573008576088588
:10855500761085A11885AC2085B42885CF3085D7C0
:108565003885DF4085EF50862158000085730286E7
:1085750027C2C5EF700F900D80E025E044A0F5C23D
:108585007F0302862DEF6401600302862D900D8026
:10859500E025E044A1F5C27F0402862D900D81E01F
:1085A500F5C27F0502862D900E117403F08079EFD8
:1085B500B4050B900D81A3E0F5C27F06806AEFB488
:1085C5000606D2C57F0180608018900E117404F0F4
:1085D5008056900E117406F0804EEFB404047F02AD
:1085E5008046900E117405F0803E900D83E0FBA34C
:1085F500E475F001124ADCA9F0FAE5C2124A92903C
:108605000D87E024FFF0900D86E034FFF0E0700266
:10861500A3E07004C2C280107F02800CD2C47F091F
:108625008006900E117401F0EFB40904C2C38036C0
:10863500900E11E0B4031C900D8874FFF5F0124AFA
:10864500C645F0600ED2C4D2C5D2C2C2C3E4900EF4
:1086550011F0FF900E11E06008C2C5D2C4C2C380FC
:0F86650005C2C302854520C7FD900D8AE0F5844C
:0186740022E3
:1088DE00900DAAEFF0900DADEBF0A3EAF0A3E9F046
:0888EE00900DABECF0A3EDF0DE
:1088F600750A00543FF50B543F605CC37440950BFA
:10890600FFE4950AFE900DB0E0FCA3E0FDC39FECEA
:108916009E50068C088D0980048E088F091283A14B
:10892600900E11E060037F0222900DACE02509F065
:10893600900DABE03508F0900DB2E0700B900DAEE7
:10894600E5088509F0124AC6C3900DB1E09509F015
:10895600900DB0E09508F0900DB0E0F508A3E0F5B5
:1089660009D3E5099400E50894004070E5099440B0
:10897600E508940050131283A1900E11E060037F66
:108986000222E4F508F50980D8900DAAE0FFA3E0DD
:10899600FCA3E0FDA3E0FBA3E0FAA3E0F9900D6ED3
:1089A600E4F074401283BD900E11E060037F022252
:1089B60074C02509F50974FF3508F508900DACE07B
:1089C6002440F0900DABE03400F0900DB2E07091D1
:0E89D600900DAE75F040124AC60289677F0010
:0189E4002270
:1093EE00900D86E4F0A304F0128511900E11E0604A
:0793FE00037F01227F002222
:10935800900E10EBF07B017A0E7910900DB0E4F0CE
:0A936800A304F0E4A3F01288DE2253
:10925F00C007900DC2E0FFA3E0900D86CFF0A3EF03
:10926F00F0D007128511900E11E060037F01227F6D
:02927F000022CB
:10937200C007900DCAE0FFA3E0900DB0CFF0A3EFBD
:0A938200F0E4A3F0D0071288DE2209
:0E902800900DE6EBF0A3EAF0A3E9F0A3EDF063
:10903600E4900DEBF0900DE6E0FBA3E0FAA3E0F977
:10904600A3E0900DD7F0900DEAE0900DD8F0E4FF84
:10905600128D9FEFB4FF0D900DEBE0FE04F0EEC312
:06906600940340D17E00DE
:01906C0022E1
:0B919A00900E09EBF0A3EAF0A3E9F04F
:1091A5007E007F007D10124CF7900E09E0FBA3E0D6
:1091B500FAA3E0F97D101287D3EF7002FF227F0139
:0191C5002287
:108EE600900D967422F0A3EFF0A37413F0124A4C7F
:108EF600900D99F0900001124A65900D9AF090003D
:108F060002124A65900D9BF0900003124A65900D7F
:108F16009CF0900004124A65900D9DF09000051299
:108F26004A65900D9EF0900006124A65900D9FF0DE
:108F36007B017A0D7996E4900DEAF07D0A0290287D
:10928100900DFD7422F0A3EFF0A37403F0A374FF1B
:10929100F07B017A0D79FDE4900DEAF07D040290F6
:0192A10028A4
:1092A200900E017422F0A3EFF0A3741CF0A374FFDC
:1092B200F07B017A0E7901E4900DEAF07D040290D0
:0192C2002883
:1092E300E4900E05F0A3EFF0A3740AF0A3EFF07B74
:0F92F300017A0E7905E4900DEAF07D04029028CF
:10491600540D5400000000000000000000000000DC
:07492600000000000000008A
:10784E0090FFFF124C99EDF090FFFF124C99EFF064
:06785E0090FFEE124C99B0
:10786400850C83850D82E4F0A3F0900012124CBDC8
:10787400E025E02454F582E4340DF583E0FEA3E032
:10788400FFFBAA06E4F9F8900012124CBDE025E0D3
:10789400240FF582E43400F583E0FEA3E0FFC3EF98
:1078A4009BFFEE9AFEE499FDE498FC850C83850D1C
:1078B40082A3A3124C36E47F40FEFDFC850C838535
:1078C4000D82A3A3E0F8A3E0F9A3E0FAA3E0FBC3CD
:1078D400124C0F400B850C83850D82E4F0A304F059
:1078E40074FF7FC0FEFDFC850C83850D82A3A3E09D
:1078F400F8A3E0F9A3E0FAA3E0FBD3124C0F500B7A
:10790400850C83850D8274FFF0A3F0850C83850DAF
:1079140082E0FEA3E0FF4E7003027BA3EFF470024B
:07792400EEF46003027A306B
:10792B00900012124CBDE025E02454F582E4340D96
:10793B00F583E0FEA3E0FFE4FCFD90000E124CBDCE
:10794B00124C36E47F01FEFDFC90000E124CBDE0A4
:10795B00F8A3E0F9A3E0FAA3E0FBC3124C0F500D20
:10796B0090000E124CBD124C420000000190001210
:10797B00124CBDE025E0240BF582E4340DF583E0D9
:10798B00FEA3E0FFE4FCFD7BFF7A0FF9F8124AF24D
:10799B0090000E124CBDE0F8A3E0F9A3E0FAA3E0CF
:1079AB00FB1290B1900006124CBD124C3690001297
:1079BB00124CBDE025E0240FF582E43400F583E0A2
:1079CB00FEA3E0FFE4FCFD900006124CBDE0F8A323
:1079DB00E0F9A3E0FAA3E0FB124AF290000A124C82
:1079EB00BD124C36E47BFF7A0FF9F890000A124C6B
:1079FB00BDE0FCA3E0FDA3E0FEA3E0FF1290B1907D
:107A0B000012124CBDE025E0240BF582E4340DF599
:107A1B0083EEF0A3EFF0900013124CBDE070030265
:027A2B007B7A64
:107A2D00027B77850C83850D82E0FEA3E064014E19
:057A3D006003027B7AEA
:107A4200900012124CBDE025E0240BF582E4340DC7
:107A5200F583E0FEA3E0FBC374FF9BFF740F9EFE61
:107A6200E49400FDE49400FCE47BFF7A0FF9F81241
:107A72004AF2900006124CBD124C36900012124C83
:107A8200BDE025E02454F582E4340DF583E0FEA345
:107A9200E0FBC374FF9BFF740F9EFEE49400FDE4C1
:107AA2009400FC90000A124CBD124C36E47F01FE99
:107AB200FDFC90000A124CBDE0F8A3E0F9A3E0FA45
:107AC200A3E0FBC3124C0F500D90000A124CBD12E2
:107AD2004C4200000001900006124CBDC083C082DF
:107AE200E0FCA3E0FDA3E0FEA3E0FF90000A124C3D
:107AF200BDE0F8A3E0F9A3E0FAA3E0FB1290B1D055
:107B020082D083124C36900012124CBDE025E02444
:107B12000FF582E43400F583E0FEA3E0FBC374FFBB
:107B22009BFF740F9EFEE49400FDE49400FC900021
:107B320006124CBDE0F8A3E0F9A3E0FAA3E0FB12C1
:107B42004AF2E47BFF7A0FF9F81290B1C374FF9FF7
:107B5200FF740F9EFE900012124CBDE025E0240B34
:107B6200F582E4340DF583EEF0A3EFF090001312EA
:087B72004CBDE06003129320FA
:107B7A00900012124CBDE0FF25E0240FF582E43498
:107B8A0000F583E0FCA3E0FDEF25E02454F582E450
:097B9A00340DF583ECF0A3EDF0CD
:067BA300900014024C9951
:06492D00410D0A00C10962
:108BFC0012945EE4900E12F0900E12E0FFC39406F5
:108C0C005018EF25E0240BF582E4340DF583E4F0E5
:108C1C00A3F0900E12E004F080DE900E127406F0B9
:108C2C00900E12E0FFC3940A501BEF25E0240BF5C5
:108C3C0082E4340DF5837407F0A374FFF0900E12E8
:108C4C00E004F080DBE4900E12F0900E12E0FFC313
:108C5C00941E502A75F014EFA42402F582E5F0342A
:108C6C00F0AF82FE7B017A0D790B900DD1E4F0A36D
:108C7C007414F0128FE2900E12E004F080CC02918A
:018C8C00EFF8
:1090F500900E0E7402F0E4A3F012945E7EF07F01F0
:109105007B017A0E790E900DD1E4F0A304F0128F55
:10911500E27EF07F007B017A0E790F900DD1E4F0AD
:0C912500A304F0128FE21291EF028BFC09
:1093200030020E20090B900047E06005D201D209FF
:0D93300022200208900047E0700204F022A5
:1093D60090F000E493F46007A3E493640260031240
:0893E60090F5E4900D0AF0225D
:1091C600900D0AE0FFC3941E501EEF75F014A42400
:1091D60002F974F035F0FA7BFF780B7C0D7D017E89
:0991E600007F14124A04C20922A0
:10913100900D0AE0C3941E502B12945E900D0AE02C
:1091410075F014A42402F582E5F034F0AF82FE7BC1
:10915100017A0D790B900DD1E4F0A37414F0128F04
:05916100E21291EF2273
:06947F00129131C2092226
:0889E500900D75EDF0A3EBF01D
:1089ED00A3E004F0900D7AEFF0A3EBF0900D75E09D
:1089FD00FF900D7AE0FED39F4003028A9975F01423
:108A0D00EEA42402F582E5F034F0AF82900D7CF0F7
:108A1D00A3EFF0900D7BE075F014A42402F582E530
:108A2D00F034F0AF82900D7EF0A3EFF0E4900D786E
:108A3D00F0A3F0900D7EE475F001124ADCAFF0FE6C
:108A4D00900D7CE0FCA3E0F5828C83E493FD128C09
:108A5D008D900D7DE004F07006900D7CE004F0909B
:108A6D000D79E004F07006900D78E004F0C3900DE0
:108A7D0079E09414900D78E0940040B71291EF9046
:108A8D000D7AE004F0A3E004F00289F9900D0AE0FC
:108A9D00FF900D76E0D39F5009A3E0C39F400312D2
:028AAD0091C670
:018AAF0022A4
:0F81E100900D8CEDF0900D8BEFF0900D8DEBF07D
:1081F000900D92EFF0A3EBF0900D8CE0FF900D92BC
:10820000E0D39F400302835CA3E075F014A4240232
:10821000F582E5F034F0AF82900D8EF0A3EFF0E43C
:10822000900D94F0A3F0900D94E0FEA3E0FFC394B2
:1082300014EE94005038900D8EE0FCA3E0F5828C93
:1082400083E493FD74272FF582E4340DF583EDF07C
:10825000900D8FE004F07006900D8EE004F0900D0C
:1082600095E004F070C0900D94E004F080B8900D9B
:1082700092E075F014A42402F582E5F034F0AF82A8
:10828000900D90F0A3EFF0900D93E075F014A424FE
:1082900002F582E5F034F0AF82900D8EF0A3EFF09E
:1082A000E4900D94F0A3F0900D8EE475F001124A65
:1082B000DCAFF0FE900D90E0FCA3E0F5828C83E44F
:1082C00093FD128C8D900D91E004F07006900D904E
:1082D000E004F0900D95E004F07006900D94E00439
:1082E000F0C3900D95E09414900D94E0940040B785
:1082F000900D92E075F014A42402F582E5F034F0BC
:10830000AF82900D90F0A3EFF0E4900D94F0A3F005
:10831000900D94E0FCA3E0FDC39414EC9400502C69
:10832000900D90E475F001124ADCAFF0FE74272D39
:10833000F582E4340DF583E0FD128C8D900D95E00F
:1083400004F070CC900D94E004F080C41291EF9092
:108350000D92E004F0A3E004F00281F8900D0AE031
:10836000FF900D8DE0FED39F5020900D8BE0FDA37C
:10837000E0C39DFDE49400FCEE7A002DFDEA3CFC98
:10838000C3ED9F7480F86C985013900D0AE0FF9035
:108390000D8BE0D39F5009A3E0C39F40031291C609
:0183A00022BA
:0B8AB000900DA0EFF0A3EDF0A3EBF0A1
:108ABB00A2AFE433A3F0C2AF129479900DA1E0FE04
:108ACB00900DA0E0FDEDFF900DA8EEF0A3EFF0E40C
:108ADB00900DA4F0900DA2E0FF900DA8E0FCA3E098
:108AEB00FD7B017A0D7927900DC2E4F0A37414F08D
:108AFB0012925F900DA9E02414F0900DA8E03400C1
:108B0B00F0900DA4E075F014A42402F974F035F084
:108B1B00FAA374FFF0A3EAF0A3E9F012945E900DB0
:108B2B00A5A3E0FAA3E0AE02FF7B017A0D792790B3
:108B3B000DD1E4F0A37414F0128FE21291EF900DAB
:108B4B00A4E004F0E0C3941E408A900046E0FF12BC
:0A8B5B009428900DA3E024FF92AFD0
:018B650022ED
:0B8B6600900DB3EFF0A3EDF0A3EBF0D7
:108B7100A2AFE433A3F0C2AF129479900DB4E0FE3A
:108B8100900DB3E0FDEDFF900DB8EEF0A3EFF0E432
:108B9100900DB7F0900DB7E0FFC3941E504C75F0E7
:108BA10014EFA42402F582E5F034F0AF82FE900DBB
:108BB100BAF0FAA3EFF0FB900DB5E0FF900DB8E02D
:108BC100FCA3E0FDA9037BFF900DCAE4F0A374149C
:108BD100F0129372900DB9E02414F0900DB8E034C6
:108BE10000F0900DB7E004F080AA900046E0FF127B
:0A8BF1009428900DB6E024FF92AF27
:018BFB002257
:03000000024000BB
:03000300025003A5
:03000B000250069A
:030013000250098F
:03001B0002500C84
:0300230002500F79
:03002B000250126E
:0300330002501563
:03003B0002501858
:0300430002501B4D
:03004B0002501E42
:0300530002502137
:03005B000250242C
:0300630002502721
:03006B0002502A16
:0300730002502D0B
:03007B0002503000
:03008300025033F5
:03008B00025036EA
:03009300025039DF
:03009B0002503CD4
:0300A30002503FC9
:10400000787FE4F6D8FD9000007F007E20E4F0A3E6
:0A401000DFFCDEFA75812102405545
:10401A00024FA8E493A3F8E493A34003F68001F2C5
:10402A0008DFF48029E493A3F85407240CC8C333A7
:10403A00C4540F4420C8834004F456800146F6DF76
:10404A00E4800B010204081020408090409AE47E2C
:10405A00019360BCA3FF543F30E509541FFEE4936B
:10406A00A360010ECF54C025E060A840B8E493A332
:10407A00FAE493A3F8E493A3C8C582C8CAC583CA5D
:10408A00F0A3C8C582C8CAC583CADFE9DEE780BE15
:014933000083
:10493400E709F608DFFA8046E709F208DFFA803E65
:1049440088828C83E709F0A3DFFA8032E309F60852
:10495400DFFA8078E309F208DFFA807088828C83BA
:10496400E309F0A3DFFA806489828A83E0A3F6086E
:10497400DFFA805889828A83E0A3F208DFFA804C48
:1049840080D280FA80C680D4806980F2803380101F
:1049940080A680EA809A80A880DA80E280CA803388
:1049A40089828A83ECFAE493A3C8C582C8CCC58300
:1049B400CCF0A3C8C582C8CCC583CCDFE9DEE780D0
:1049C4000D89828A83E493A3F608DFF9ECFAA9F04F
:1049D400EDFB2289828A83ECFAE0A3C8C582C8CCA5
:1049E400C583CCF0A3C8C582C8CCC583CCDFEADEBE
:1049F400E880DB89828A83E493A3F208DFF980CC20
:104A040088F0EF60010E4E60C388F0ED2402B40418
:104A14000050B9F582EB2402B4040050AF232345BF
:064A240082239049847317
:104A2A00C2D530F707B2D563F0FF05F030E70CB214
:104A3A00D5F4048463F0FF05F080018430D502F4D4
:024A4A00042244
:104A4C00BB010689828A83E0225002E722BBFE0268
:094A5C00E32289828A83E493229B
:104A6500BB010CE58229F582E5833AF583E0225006
:104A750006E92582F8E622BBFE06E92582F8E22250
:0D4A8500E58229F582E5833AF583E493226A
:104A9200BB010689828A83F0225002F722BBFE0103
:024AA200F322FD
:104AA400F8BB010DE58229F582E5833AF583E8F048
:104AB400225006E92582C8F622BBFE05E92582C8F4
:024AC400F222DC
:104AC600C5F0F8A3E028F0C5F0F8E582158270027B
:064AD6001583E038F02218
:104ADC00A3F8E0C5F025F0F0E5821582700215838D
:064AEC00E0C838F0E822EA
:104AF200E88FF0A4CC8BF0A42CFCE98EF0A42CFC63
:104B02008AF0EDA42CFCEA8EF0A4CDA8F08BF0A4E0
:104B12002DCC3825F0FDE98FF0A42CCD35F0FCEB3F
:104B22008EF0A4FEA9F0EB8FF0A4CFC5F02ECD3904
:0F4B3200FEE43CFCEAA42DCE35F0FDE43CFC2271
:104B410075F008758200EF2FFFEE33FECD33CDCC2B
:104B510033CCC58233C5829BED9AEC99E5829840AE
:104B61000CF582EE9BFEED9AFDEC99FC0FD5F0D68B
:104B7100E4CEFBE4CDFAE4CCF9A88222B800C1B9B5
:104B81000059BA002DEC8BF084CFCECDFCE5F0CBF3
:104B9100F97818EF2FFFEE33FEED33FDEC33FCEB2C
:104BA10033FB10D703994004EB99FB0FD8E5E4F9E7
:104BB100FA227818EF2FFFEE33FEED33FDEC33FCD4
:104BC100C933C910D7059BE99A4007EC9BFCE99AC8
:104BD100F90FD8E0E4C9FAE4CCFB2275F010EF2F0D
:104BE100FFEE33FEED33FDCC33CCC833C810D7070D
:104BF1009BEC9AE899400AED9BFDEC9AFCE899F848
:0E4C01000FD5F0DAE4CDFBE4CCFAE4C8F922DA
:1090B100C2D5E830E70FB2D5E4C39BFBE49AFAE4EA
:1090C10099F9E498F8EC30E717B2D51290E7124B12
:1090D1007DE4C39BFBE49AFAE499F9E498F88003F0
:1090E100124B7D30D50DE4C39FFFE49EFEE49DFD50
:0490F100E49CFC22DD
:104C0F00EB9FF5F0EA9E42F0E99D42F0EC6480C81C
:064C1F0064809845F022BC
:104C2500EB9FF5F0EA9E42F0E99D42F0E89C45F0E5
:014C3500225C
:0C4C3600ECF0A3EDF0A3EEF0A3EFF022F1
:104C4200A8828583F0D083D082124C59124C59121B
:104C52004C59124C59E473E493A3C583C5F0C58340
:104C6200C8C582C8F0A3C583C5F0C583C8C582C8BC
:014C7200221F
:104C7300D083D082F8E4937012740193700DA3A3D0
:104C830093F8740193F5828883E4737402936860E4
:064C9300EFA3A3A380DFE4
:104C9900E50D2582F582E50C3583F583B50C048590
:104CA900820D2210AF0685820DF50C2285820DF545
:044CB9000CD2AF2248
:0D4CBD00E50D2582F582E50C3583F5832297
:104CCA00EC8EF0A4CCC5F0CCCDF8EFA4CEC5F02D77
:104CDA00FDE43CFCE8A42EC8C5F03DFDE43CFCEF35
:0D4CEA00A4FFE5F028FEE43DFDE43CFC22C3
:104CF700EF4E6012EF60010EEDBB010B89828A83D4
:104D0700F0A3DFFCDEFA2289F05007F709DFFCA9E0
:0C4D1700F022BBFEFCF309DFFCA9F02237
:00000001FF
